:100000008B285630A7002708A600A60B0528080055
:100010002B30A7002708A600A60B0C280800A30079
:100020000830A400A30985140120A30C031C1A287E
:1000300085141B2885100120A40B1528851001208C
:1000400000000800851D22280820851D2228083070
:10005000A400A3010120A30CA317851DA313A40BC7
:100060002A28A30923080800FF010630831681000F
:10007000831281012730FF076400831201087F0685
:10008000031943283D28FF037F0A0319FF037F0854
:100090007F04031D3A280800FF0000000000FF0B4A
:1000A0004D28080005116D30A3000000A30B552852
:1000B0000000000005150800A3000830A400051189
:1000C0000000000000000000000000000000000030
:1000D0000000000000000000000000000000A30C71
:1000E000031C752800000515782805110000000084
:1000F0000000000000000000000000000000000000
:1001000000000000A40B6F280000000000000000A9
:10011000000005150800831285010730990008309A
:100120008316850083128312051542300F2022208A
:10013000A0002008503A0319A428023A0319B32852
:10014000183A0319B528C3282220A1005220A20181
:10015000210822020318B2282220A00020085C20D7
:10016000A20AA828C3289328C3282220A100A201FC
:10017000210822020318C2282220A00020085C20A7
:08018000A20AB828C328972841
:02400E000200AE
:00000001FF
